:1000000012C024C023C022C021C020C01FC01EC0F7
:100010001DC01CC01BC01AC019C018C017C016C014
:1000200015C014C013C011241FBECFE5D4E0DEBF3D
:10003000CDBF10E0A0E6B0E0EAEDFCE002C0059024
:100040000D92A236B107D9F731D545C6D9CFBF92A7
:10005000CF92DF921F93CF93DF93DC01CB01142F5C
:10006000E901E3E1FCE00F921F927EEF65E659EAB9
:1000700040E8D92EC82EBA2E212F1D2E0C2E099500
:100080002131F9F71F900F90DF91CF911F91DF90F1
:10009000CF90BF900895BF92CF92DF921F93CF93DE
:1000A000DF93DC01CB01142FE901E3E9FFE00F92BC
:1000B0001F927EEF65E659EA40E8D92EC82EBA2E87
:1000C000212F1D2E0C2E09952131F9F71F900F902D
:1000D000DF91CF911F91DF90CF90BF900895CF9384
:1000E000DF93FA01E9012134310510F0C0E4D0E0DA
:1000F000AB01BC01407C9E01CF01CFD4CE01DF918A
:10010000CF9108952F923F924F925F926F927F927C
:100110008F929F92AF92BF92CF92DF92EF92FF9217
:100120000F931F93CF93DF934A01E90121343105E7
:1001300010F0C0E4D0E01E01369427946B017C01DE
:1001400020ECC222D40180E090E060E070E08215F3
:100150009305B9F0F601E819F909EA0FFB1F25919B
:1001600034914D915D912417350709F071E0409568
:100170005095422B532B4F3F5F4F09F061E00196A2
:10018000E6CF772351F1662339F020E030E043E0F9
:10019000C701B601F801099526013701A12CB12C40
:1001A000A214B30491F0F401219131914F0141E087
:1001B000C301B201F8010995F2E04F0E511C611C18
:1001C000711C2FEFA21AB20AEBCF20E030E045E01D
:1001D000C701B601F801099502C0C0E0D0E0CE0128
:1001E000DF91CF911F910F91FF90EF90DF90CF9013
:1001F000BF90AF909F908F907F906F905F904F9047
:100200003F902F9008950F931F93682F70E080E028
:1002100090E048E08B019C0136952795179507954E
:1002200060FF0BC0C901B80150E2652753E875278C
:1002300058EB85275DEE952702C0C901B8014150F2
:1002400049F71F910F910895CF92DF92EF92FF929D
:10025000C72ED82EE92EFF24842F8627D4DF6C25C5
:100260007D258E259F25FF90EF90DF90CF900895FC
:1002700028E088E190E00FB6F894A89581BD0FBE04
:1002800021BDA895F894D4E0CEE52CE0299320E098
:10029000299314BEFFCF8FEF089563C0ADC088C00F
:1002A00087C086C085C084C083C082C081C080C032
:1002B0007FC07EC07DC07CC07BC07AC079C078C062
:1002C0007E3FF9F76536F9F7593AF9F74038F9F70B
:1002D000EC2DFD2DB7B6B0FCFDCF27BFE895B7B626
:1002E000B0FCFDCF21E1B7B6B6FCF4CF089555536D
:1002F000422076302E39372E312C206279205374EB
:10030000657068616E2042616572776F6C6600008F
:1003100009021200010100803209040000000000FF
:10032000000012011001FF000008C016DC050201E8
:10033000010200010E0355005300420061007300EA
:1003400070001C037700770077002E0066006900BC
:100350007300630068006C002E00640065000403F5
:10036000090411241FBECFE5D4E0DEBFCDBF24B702
:10037000D4E0CEE539913C30399109F03FEF30932C
:100380009B0020939A0010E0A0E6B0E0EAEFFFE1C6
:1003900002C005900D92A636B107D9F720E0A6E677
:1003A000B0E001C01D92AA39B207E1F783D170C352
:1003B00074CFDC018FEF9FEF332715C02D912827D5
:1003C000722F22952727822F269526952827239559
:1003D0002270321777952795822F8927972F769548
:1003E000279597278227615048F780959095089523
:1003F000E0DF8D939D930895CF93CFB7CF93DF9395
:10040000C395869BE9F7869B0BC0869B09C0869B9C
:1004100007C0869B05C0869B03C0869B01C089C020
:100420006F93C0917D00DD27CC57DF4F2F9365E59B
:10043000869B03C02F916F91E6CF0F931F934F932D
:1004400020E040E15F9300B3047406FB27F93F937B
:1004500050E03BE039C0147440642F77012F5F5F98
:100460001EC0406810B314742F7752501FC04064F0
:1004700000B32F770474D1F15F5F00C023C04062E6
:1004800010B32F77147491F15F5F00C025C004741E
:100490001027515012F45D5F0000115027952C3F3A
:1004A00010B3C8F614740127015027952C3FC8F6E5
:1004B0004227499300B3047410274F7311502795B6
:1004C0002C3FA8F64695469510B3147479F0012791
:1004D000015027952C3F98F66B5A60F3315000B3CA
:1004E000B0F600C010E41ABF002717C03B5031958A
:1004F000C31BD04010E41ABF0881033CF9F00B3451
:10050000E9F020917B001981110F1213EDCF09360C
:1005100051F10D3211F0013E39F7009382003F9105
:100520005F914F911F910F912F916F91CAB7C6FDA7
:1005300067CFDF91CF91CFBFCF91189520918200E7
:10054000222369F310918000112339F534303AF1F8
:100550003093800020937C0010917D003BE0311BA4
:1005600030937D001CC0009180000130B4F40AE596
:100570003091610034FD14C000936100C0E7D0E009
:1005800013C0052710E000C0000002BB1AC00527F9
:1005900010E0221F1DC010E021C04AE502C032ED6C
:1005A000432FC4E1D0E032E011B31464969A02B351
:1005B00011BB54E420E865E320FF052702BB279523
:1005C00017951C3FF0F66695B8F7B1F720FF0527A1
:1005D00002BB279517951C3FD0F62795179517FF57
:1005E000052700001C3F02BBB0F629913A9519F788
:1005F0000B7B10918100110FC651D04002BB11F04E
:1006000010937B0010E41ABF006411B31B7B402FD2
:100610004B7B54E05A95F1F702BB11BB42BB7FCF35
:10062000F8948E9A97981BBE15BEF1E0FBBF1BBED7
:1006300034C2FC013381932F4481842F22812033E3
:1006400039F44370E42FF0E0EE59FF4F80810895B4
:10065000283529F431110EC0E1E0F0E006C0203564
:1006600071F4311125C0E0E0F0E089E0809357009B
:10067000849108953830E1F4E3E0F0E0F6CF2032E1
:1006800021F4FC01EE0FFF1F06C0283231F4FC01FB
:10069000EE0FFF1F319684910895203A09F4E3C1CB
:1006A000203C19F46581E7D103C02F3F09F411EF15
:1006B00080E0089511BA80E882BB81E08BBF82E0C0
:1006C0008BBF84E031978040E9F780919A00877F63
:1006D00021F480919B00882311F08799A1DF1EEF00
:1006E00014BE85B7826085BF8BB780648BBF8E9A3E
:1006F00080E131978040E9F78E98789400918000EE
:10070000035007FD2BC180917D00CCE0D0E0C81BD9
:10071000D109CC57DF4F80917C008D3209F0B5C0F4
:10072000083009F019C183EC809370008AE580934A
:10073000610010926F004881842F80763981882370
:1007400099F186E690E090937F0080937E003330AD
:1007500031F4CE016EDF8093690024E08CC0353027
:10076000F9F03A30E9F08CEF830F863098F48A8103
:100770009B8190936E0080936D00393099F08E814B
:1007800080936C008D81827080936B0030936A003F
:100790002FEF6BC0323011F41E7F04C0116002C015
:1007A00021E069C020E067C08A8110927900311190
:1007B00006C010927A0089E790E022E050C0353000
:1007C00019F4809381003DC03630A9F59B819130AA
:1007D00019F488E898E104C0923041F486E798E182
:1007E00090937F0080937E0022E121C09330F1F44A
:1007F000811108C084EC98E190937F0080937E0083
:1008000024E015C0813041F488EA98E190937F009C
:1008100080937E002CE10BC0823041F48AE998E19C
:1008200090937F0080937E002EE001C020E080E462
:1008300080936F0018C0383079F0393031F48093EC
:10084000830089E790E020E00AC021E03A3009F017
:1008500020E089E790E003C083E890E021E09093F6
:100860007F0080937E002F3F31F447FD2E8180E88A
:1008700080936F0007C08F81811104C08E81821721
:1008800008F4282F2093600067C080916F0087FFD5
:1008900063C080916C00801708F4082F801B809340
:1008A0006C00DD24D3948111D12C80916A008730B3
:1008B000C0F0CC2EEC2EFD2E8E2D8C19801708F05A
:1008C00048C0D7016D917D0180916D0090916E00BF
:1008D0009C012F5F3F4F30936E0020936D00CBD073
:1008E000EBCF80916B00E0916D00F0916E00DE0126
:1008F00000FD0395025048F1F83138F522D0F89404
:100900000D901D9021E017D02E2F2E5F2F7331F008
:10091000DD2079F0882369F0003059F423E00BD012
:1009200010D025E008D00DD007B606FE02C021E1A8
:1009300002D03296DFCFF89427BFE895112478943F
:10094000089507B600FCFDCF0895F0936E00E09384
:100950006D00D110109260001092800080916100B3
:1009600084FF6BC0809160008F3F09F466C0082F40
:10097000893008F008E0801B80936000809170004F
:1009800098E8892780937000002309F44AC0809179
:100990006F0087FF28C080916C00801708F4082F33
:1009A000801B80936C00D0906A00C1E7D0E081E7A3
:1009B00090E02C2F281B2017A0F5E0906D00F09000
:1009C0006E00B6E0BD1518F4C7014DD002C0F701A6
:1009D000849188832196FFEFEF1AFF0AF0926E0050
:1009E000E0926D00E4CFE0917E00F0917F0086FF01
:1009F0000BC081E790E0DC0124912D933196202FEC
:100A0000280F2A13F9CF09C081E790E0DC0121917A
:100A10002D93202F280F2A13FACFF0937F00E09315
:100A20007E00602F81E790E0E3DC0C5F0C3019F072
:100A30008FEF809360000093610084E190B3947421
:100A400031F48150D9F71092810010927B0010315F
:100A500018F08799105104C0123010F0879B125083
:100A600011114CCE3BCEE199FECF9FBB8EBBE09ADD
:100A700099278DB30895262FE199FECF9FBB8EBB9A
:100A80002DBB0FB6F894E29AE19A0FBE0196089535
:100A9000F894FFCFFF5A1E930700FA01DC0102C051
:100AA00005900D9221503040D8F70895CF93DF93F1
:100AB000CDB7DEB7C054D1090FB6F894DEBF0FBE74
:100AC000CDBF84B714BE98E10FB6F89491BD11BCA8
:100AD0000FBE8E9AF8948F98979AB89AB99A8D9A71
:100AE0008B9A959A83FDEDC0C0906000D090610014
:100AF000E12CF12C6FEF7FEFCB01F701EC0DFD1D29
:100B00004491A2DB2FEFE21AF20AE114E8E0FE06BC
:100B1000A1F76A3C7D4987439D4809F0AEC0198220
:100B200080E090E0F601E80FF91F45915491FC0137
:100B3000F85E259134914217530719F081E08983BB
:100B400005C00296811528E0920761F78981882304
:100B500009F493C016E2C12E18E1D12EE12CF12C3C
:100B6000B701A601407C20E430E0CE01019695DF7C
:100B7000C701B6016652794F8F4F9F4F07E210E0D1
:100B800020E430E0AE014F5F5F4FBCDA80E4C80E76
:100B9000D11CE11CF11CE6E2CE16E9E1DE06E1041F
:100BA000F104F1F6C12CB8E1DB2EE12CF12C560159
:100BB000F8E1BF1A40E450E06FEF70E0CE0101961B
:100BC00083D040916000509161004A0D5B1D662703
:100BD00057FD6095762F20E430E0CE0101965DDF71
:100BE0000BE410E020E430E0AE014F5F5F4FC7013F
:100BF000B60188DA20E4C20ED11CE11CF11C80E8A9
:100C0000C81689E1D806E104F10489F6E12CA8E0D0
:100C1000FA2EEA18FB0840E450E06FEF70E0CE01D6
:100C2000019652D09701E1E4EE16F10410F020E4B1
:100C300030E040916000509161004A0D5B1D6627D5
:100C400057FD6095762FCE01019627DFB501785EBE
:100C500080E090E007E210E020E430E0AE014F5F7A
:100C60005F4F50DAF0E4AF0EB11C20E4E21AF10855
:100C7000A11488E0B80678F2C19AC09A20E630E064
:100C8000C901880F991F820F931F0596009779F06D
:100C9000EFE9FFE03197F1F700C00000879905C048
:100CA0009398879BFECF20E630E00197EFCF82B389
:100CB00098E0892782BB215031092115310501F7C0
:100CC000D7DA939AA895FECFDC0101C06D9341500D
:0A0CD0005040E0F70895F894FFCFBC
:020CDA009A027C
:00000001FF
